:020000040000FA
:1000000000308A0004280000840183131F30830518
:10001000623083168F000F081F129F121B08803951
:100020009B0007309C001F129F121B088039033869
:100030009B001F1383121F179F1783169F1783128E
:100040001F149412831606118614061201308312AF
:1000500094000030831694000108C73908388100E5
:10006000831290010030F800920000308316920055
:1000700007309C00050885000330F700F70B3E2889
:0C0080001C0883120D1383169D01630001
:04400E00393FFF3FF8
:00000001FF
